:100000000C942A000C9445000C9445000C94450077
:100010000C9445000C94F7010C9424020C944C02AF
:100020000C9445000C9480010C9445000C94450000
:100030000C9445000C9445000C946E030C94450000
:100040000C9445000C9445000C9445000C9445001C
:100050000C94450011241FBECFE5D4E0DEBFCDBF18
:1000600010E0A0E6B0E0EEE2FEE002C005900D92E6
:10007000A239B107D9F710E0A2E9B0E001C01D92A2
:10008000AA3EB107E1F70C94AD000C940000CF93A9
:10009000DF93CDB7DEB7E7E3F0E08FE18083E4E301
:1000A000F0E08CEF8083E1E3F0E084E08083E2E342
:1000B000F0E088E38083DF91CF910895CF93DF93C1
:1000C000CDB7DEB721970FB6F894DEBF0FBECDBF18
:1000D000F89480E29EE49093E7008093E600198212
:1000E0002FC08981482F552789819927880F991F0B
:1000F000FC01E355FF4F808191819C0128513C4FC9
:10010000CA01880F991FFC01EA52FF4F31832083F7
:100110002091E6003091E70089819927880F991F87
:10012000FC01EA52FF4F80819181A901481B590BC4
:10013000CA019093E7008093E60089818F5F8983ED
:100140008981883070F2789421960FB6F894DEBFDA
:100150000FBECDBFDF91CF910895CF93DF93CDB781
:10016000DEB727970FB6F894DEBF0FBECDBF0E9453
:1001700047000E945E010E9460030E94AF0310923C
:10018000D4008BE093E09093A8008093A70089E5CA
:1001900093E09093AA008093A900789480919600B0
:1001A0008823E1F3109296000E9442060E94970471
:1001B00000C080919800813041F4109298008091A5
:1001C000D400882311F40E945E0080919600813053
:1001D00019F5109296001A821CC080E690E00E94E9
:1001E000E9038A8199270E94330487E690E00E9400
:1001F000E9038A819927880F991FFC01EA52FF4F72
:10020000808191810E9433040E9424048A818F5F3F
:100210008A838A81893008F380919500813049F67C
:10022000109295008091D5008595992787FD90952E
:1002300090939A00809399002091990030919A00B0
:10024000CE0103964AE050E0BC01C9010E94D206EB
:10025000CE010396DC01FD0101900020E9F7319702
:10026000CF018A1B9B0B89836AE080E00E941E06F7
:100270008AE690E00E94C0059DE08981292F281B15
:10028000822F682F80E00E941E06CE0103960E94F6
:10029000C0058FCFCF93DF93CDB7DEB7F894E9E5F4
:1002A000F0E089E180837894DF91CF910895CF9336
:1002B000DF93CDB7DEB7DF91CF910895CF93DF9372
:1002C000CDB7DEB7E3E5F0E082E08083EFE4F0E075
:1002D0001082EEE4F0E082E08083EAE4F0E084EF74
:1002E00091E091838083E8E4F0E080ED97E09183F2
:1002F0008083E9E5F0E089E18083DF91CF91089583
:100300001F920F920FB60F9211242F933F934F938A
:100310005F936F937F938F939F93AF93BF93EF936D
:10032000FF93CF93DF93CDB7DEB780919E008F5FB1
:1003300080939E0080919E00883021F40E9489065F
:1003400010929E008091D3008F5F8093D3008091A4
:10035000D3008834C9F581E0809397001092D300D0
:1003600080919D008F5F80939D0080919D008530DE
:1003700029F410929D0081E08093980080919B0069
:100380008F5F80939B0080919B00843641F4109294
:100390009B0081E08093940081E08093960080919F
:1003A0009B00823319F481E08093960080919C0039
:1003B0008F5F80939C0080919C008A3029F410927A
:1003C0009C0081E080939500DF91CF91FF91EF91A8
:1003D000BF91AF919F918F917F916F915F914F915D
:1003E0003F912F910F900FBE0F901F9018951F9265
:1003F0000F920FB60F9211242F933F934F935F9359
:100400006F937F938F939F93AF93BF93EF93FF93DC
:10041000CF93DF93CDB7DEB7E091A700F091A800AE
:100420000995DF91CF91FF91EF91BF91AF919F918E
:100430008F917F916F915F914F913F912F910F908D
:100440000FBE0F901F9018951F920F920FB60F922C
:1004500011248F93AF93BF93EF93FF93CF93DF93C9
:10046000CDB7DEB7A2E3B0E0E2E3F0E080818B7FBE
:100470008C93A8E3B0E0E8E3F0E080818F7E8C937A
:10048000DF91CF91FF91EF91BF91AF918F910F903D
:100490000FBE0F901F9018951F920F920FB60F92DC
:1004A00011242F933F938F939F93AF93BF93EF9319
:1004B000FF93CF93DF93CDB7DEB72297DEBFCDBFDB
:1004C000A2E3B0E0E2E3F0E0808184608C93ECE4AE
:1004D000F0E011821082A8E4B0E0809192009927A8
:1004E000880F991FFC01EA52FF4F8081918111967C
:1004F0009C938E9380919200882339F4A8E3B0E016
:10050000E8E3F0E0808180618C9380919200282F55
:1005100033273A83298389819A8182309105C1F1F9
:1005200029813A812330310554F489819A810097D9
:1005300089F029813A8121303105D9F04EC0898175
:100540009A818330910599F129813A8124303105CE
:10055000E9F143C0A8E3B0E0E8E3F0E08081806126
:100560008C93A8E3B0E0E8E3F0E0808181608C93B5
:1005700034C0A8E3B0E0E8E3F0E080818E7F8C93A4
:10058000A8E3B0E0E8E3F0E0808182608C9325C0CE
:10059000A8E3B0E0E8E3F0E080818D7F8C93A8E3EE
:1005A000B0E0E8E3F0E0808184608C9316C0A8E3BB
:1005B000B0E0E8E3F0E080818B7F8C93A8E3B0E0CB
:1005C000E8E3F0E0808188608C9307C0A8E3B0E0A6
:1005D000E8E3F0E08081877F8C93809192008F5FC9
:1005E0008093920080919200893010F010929200D6
:1005F0002296F894DEBFCDBFDF91CF91FF91EF91AE
:10060000BF91AF919F918F913F912F910F900FBE0E
:100610000F901F901895CF93DF93CDB7DEB78091E1
:100620009F009091A0000097B1F4E6E4F0E0808193
:1006300091819093A6008093A500AEE4B0E0EEE433
:10064000F0E080818F7B8C9381E090E09093A0001C
:1006500080939F002BC0E6E4F0E08081918190932D
:10066000A4008093A300AEE4B0E0EEE4F0E080816B
:1006700080648C932091A3003091A4008091A50008
:100680009091A600A901481B590BCA019093A200A2
:100690008093A1001092A00010929F008091A10071
:1006A0009091A2009093E9008093E800DF91CF91B0
:1006B0000895CF93DF93CDB7DEB7DF91CF91089543
:1006C000CF93DF93CDB7DEB7E7E2F0E01082E6E24A
:1006D000F0E08FEE8083DF91CF9108951F920F920B
:1006E0000FB60F9211242F933F938F939F93EF9305
:1006F000FF93CF93DF93CDB7DEB7E6E2F0E0108251
:10070000809193009927E4E2F0E020813181880F05
:10071000991FFC01E355FF4F3183208380919300A3
:100720008F5F8093930080919300883010F0109237
:100730009300E7E2F0E0809193008083E6E2F0E04E
:100740008FEE8083DF91CF91FF91EF919F918F91F9
:100750003F912F910F900FBE0F901F901895CF9340
:10076000DF93CDB7DEB7E9E2F0E080E18083E0E43B
:10077000F0E01082EAE2F0E088E18083E0E4F0E07B
:1007800086E88083EBE2F0E082EC8083DF91CF911A
:100790000895CF93DF93CDB7DEB721970FB6F894C6
:1007A000DEBF0FBECDBF8983EBE2F0E080819927E9
:1007B000807290700097C1F3ECE2F0E08981808351
:1007C00021960FB6F894DEBF0FBECDBFDF91CF915B
:1007D0000895CF93DF93CDB7DEB726970FB6F89481
:1007E000DEBF0FBECDBF9E838D838D819E81DC01D8
:1007F000FD0101900020E9F73197CF018A1B9B0B87
:100800009C838B831A8219820FC029813A818D8142
:100810009E81F901E80FF91F80810E94C903898137
:100820009A8101969A83898329813A818B819C815F
:100830008217930750F726960FB6F894DEBF0FBEC7
:10084000CDBFDF91CF910895CF93DF93CDB7DEB7C2
:1008500080916E000E94C90380916F000E94C903BD
:10086000DF91CF910895CF93DF93CDB7DEB7669731
:100870000FB6F894DEBF0FBECDBF9E8B8D8B8D89DA
:100880009E894AE050E09E012F5F3F4FB9010E94D0
:10089000D206CE0101960E94E90366960FB6F8943F
:1008A000DEBF0FBECDBFDF91CF910895CF93DF9311
:1008B000CDB7DEB722970FB6F894DEBF0FBECDBF1F
:1008C0008A8387E089831FC08A81482F55278981C1
:1008D000282F332727FD309581E090E0022E02C0BB
:1008E000880F991F0A94E2F7842395231816190696
:1008F00024F481E30E94C90303C080E30E94C9037A
:1009000089818150898389818823F4F680916E00E2
:100910000E94C90380916F000E94C90322960FB6FE
:10092000F894DEBF0FBECDBFDF91CF910895CF9376
:10093000DF93CDB7DEB70E94BA0463E080E00E9487
:100940001E0680E790E00E94C00562E081E00E9400
:100950001E068BE790E00E94C005E0E3F0E0808196
:100960009927807290700097C1F70E94BA04DF91B6
:10097000CF910895CF93DF93CDB7DEB781E00E948A
:10098000F505DF91CF910895CF93DF93CDB7DEB713
:1009900026970FB6F894DEBF0FBECDBF9E838D8322
:1009A0008AE090E09C838B831CC082E390E09A8372
:1009B00089830EC08D819E8101979E838D838D8159
:1009C0009E810097B9F789819A8101979A838983DB
:1009D00089819A81009799F78B819C8101979C83EB
:1009E0008B838B819C81009701F726960FB6F89434
:1009F000DEBF0FBECDBFDF91CF910895CF93DF93C0
:100A0000CDB7DEB721970FB6F894DEBF0FBECDBFCE
:100A100089838981992781709070882341F0A5E3AB
:100A2000B0E0E5E3F0E0808180618C9307C0A5E34E
:100A3000B0E0E5E3F0E080818F7E8C938981992797
:100A400082709070009741F0A5E3B0E0E5E3F0E03C
:100A5000808180628C9307C0A5E3B0E0E5E3F0E01D
:100A600080818F7D8C938981992784709070009705
:100A700041F0A5E3B0E0E5E3F0E0808180648C9391
:100A800007C0A5E3B0E0E5E3F0E080818F7B8C93C5
:100A90008981992788709070009741F0A5E3B0E0B4
:100AA000E5E3F0E0808180688C9308C0A5E3B0E0C6
:100AB000E5E3F0E090818FE789238C9321960FB6D0
:100AC000F894DEBF0FBECDBFDF91CF910895CF93D5
:100AD000DF93CDB7DEB7A5E3B0E0E5E3F0E08081DA
:100AE00084608C9381E090E00E94C404A5E3B0E0B0
:100AF000E5E3F0E080818B7F8C93DF91CF910895C7
:100B0000CF93DF93CDB7DEB722970FB6F894DEBF51
:100B10000FBECDBF8A838A8182958F708983898138
:100B20000E94FE040E9467058A810E94FE040E94C2
:100B3000670522960FB6F894DEBF0FBECDBFDF91DA
:100B4000CF910895CF93DF93CDB7DEB721970FB63E
:100B5000F894DEBF0FBECDBF8983A5E3B0E0E5E327
:100B6000F0E0808188608C9389810E9480052196C5
:100B70000FB6F894DEBF0FBECDBFDF91CF910895C1
:100B8000CF93DF93CDB7DEB724970FB6F894DEBFCF
:100B90000FBECDBF9C838B838B819C81DC01FD01CB
:100BA00001900020E9F73197CF018A1B9B0B8A83C4
:100BB00019820EC0898199279C018B819C81F90142
:100BC000E80FF91F80810E94A20589818F5F8983C8
:100BD00099818A81981770F324960FB6F894DEBF36
:100BE0000FBECDBFDF91CF910895CF93DF93CDB7E7
:100BF000DEB721970FB6F894DEBF0FBECDBF898355
:100C000081E090E00E94C404A5E3B0E0E5E3F0E0F9
:100C10008081877F8C9389810E948005A5E3B0E065
:100C2000E5E3F0E0808188608C9321960FB6F8941C
:100C3000DEBF0FBECDBFDF91CF910895CF93DF937D
:100C4000CDB7DEB723970FB6F894DEBF0FBECDBF8A
:100C50008A836B838A81882319F48B8180588983E6
:100C60008A81813019F48B818054898389810E9423
:100C7000F50523960FB6F894DEBF0FBECDBFDF910A
:100C8000CF910895CF93DF93CDB7DEB781E090E0A9
:100C90000E94C404A5E3B0E0E5E3F0E08081877F33
:100CA0008C9383E00E94FE040E94670585E090E03B
:100CB0000E94C40483E00E94FE040E94670581E054
:100CC00090E00E94C40483E00E94FE040E94670535
:100CD00082E00E94FE040E94670581E090E00E948D
:100CE000C40488E20E94F5058EE00E94F50581E0CB
:100CF0000E94F50588E890E00E94C0056AE081E066
:100D00000E941E068DE890E00E94C005DF91CF9101
:100D10000895CF93DF93CDB7DEB721970FB6F89440
:100D2000DEBF0FBECDBF1982E0E3F0E080819927DE
:100D300080719070009711F081E08983E0E3F0E02A
:100D40008081992788709070009721F0898193E0C5
:100D500089278983998180916900292F281B822FF7
:100D600089838981992787FD909581709070882368
:100D700081F080916900982F8981890F80936900A3
:100D80008981982F92708091D500890F815080932E
:100D9000D50021960FB6F894DEBF0FBECDBFDF9110
:100DA000CF910895FB019F01E8944230C4F0453291
:100DB000B4F44A3029F497FB1EF4909581959F4F27
:100DC000642F77270E940307805D8A330CF0895DCA
:100DD0008193CB010097A1F716F45DE25193108245
:100DE000C9010C94F306DC01FC0101900020E9F735
:100DF0003297AE17BF0730F47C91608170833197D2
:100E00006D93F7CF0895AA1BBB1B51E107C0AA1F22
:100E1000BB1FA617B70710F0A61BB70B881F991F9B
:0E0E20005A95A9F780959095BC01CD010895D3
:100E2E004B2000000000003D0001202020000D0A94
:100E3E004550492D54657374657200566572736919
:100E4E006F6E20302E3263006875687500416B6BD3
:020E5E0075001D
:00000001FF
